:1000000045C0000053C0000051C000004FC00000B8
:100010004DC000004BC0000049C0000047C00000B8
:1000200045C0000043C0000041C000003FC00000C8
:1000300071C100003BC0000039C0000037C00000A3
:1000400035C0000033C0000031C000002FC00000E8
:100050002DC000002BC0000029C0000027C00000F8
:1000600025C0000023C0000021C000001FC0000008
:100070001DC000001BC0000019C0000017C0000018
:1000800015C0000013C0000011C0000011241FBEE5
:10009000CFEFD0E1DEBFCDBF21E0A0E0B1E001C0F5
:1000A0001D92A330B207E1F770D060C1A9CF8FEFE6
:1000B00081BB9FE39ABB8BBB1CBEF8948DE08EBDC9
:1000C00088E09DE39BBD8ABD84E086BF15BE10928B
:1000D0006A0019BE80E187BF78940895843041F1A9
:1000E00048F48130C9F0A0F08230D1F0833009F0BB
:1000F0004AC01AC0873041F130F48530E9F08630CB
:1001000009F041C01DC0883019F18930E1F524C0E3
:10011000613031F59FE337C0613021F596E033C09F
:10012000613011F59BE52FC0613001F59FE42BC0D4
:100130006130F1F496E627C06130E1F49DE623C01A
:100140006130D1F49DE71FC06130C1F497E01BC05E
:100150006130B1F49FE717C06130A1F49FE613C08E
:1001600090E411C099EF0FC094E20DC090EB0BC06A
:1001700099E109C092E907C092E005C098EF03C079
:1001800090E001C090E9892F089591DF1BBA8FEFAD
:1001900082BBCDEC0F2EFFEDDF2EF02D0F2EFFEEEC
:1001A000EF2EF02D0F2EF7EFFF2EF02D0BEF1DEFA2
:1001B000DEEFCE9917C02FEF83EC99E021508040FD
:1001C0009040E1F700C00000809101018B3330F4D2
:1001D0008F5F809301011092000104C01092010111
:1001E00010920001CF9917C02FEF83EC99E02150B6
:1001F00080409040E1F700C000008091020187310B
:1002000030F48F5F809302011092000104C01092BD
:10021000020110920001809100018C9F912D112408
:10022000969596959695990F292F220F220F920F4A
:1002300060E0891B53DF82BBDBBA8FE99FE0019747
:10024000F1F700C00000809100018C9F812D1124E6
:1002500060E086958695869541DF82BBEBBA8FE993
:100260009FE00197F1F700C00000809101018C9F91
:10027000912D1124969596959695990F292F220FD9
:10028000220F920F60E0891B29DF82BBFBBA8FE946
:100290009FE00197F1F700C00000809101018C9F61
:1002A000812D112460E086958695869517DF82BBA7
:1002B0000BBB8FE99FE00197F1F700C00000809130
:1002C00002018C9F912D1124969596959695990FE4
:1002D000292F220F220F920F60E0891BFFDE82BBC5
:1002E0001BBB8FE99FE00197F1F700C000008091F0
:1002F00002018C9F812D112460E08695869586955C
:10030000EDDE82BBDBBB8FE99FE00197F1F700C018
:1003100000004FCF1F920F920FB60F9211248F93B0
:10032000809100018F5F8C3319F08093000107C02A
:1003300010920001809101018F5F809301018091F3
:1003400001018C3339F410920101809102018F5F19
:100350008093020180910201883110F01092020115
:100360008F910F900FBE0F901F901895F894FFCFAC
:00000001FF
